:020000002EC010
:10000200FECFFDCFFCCFFBCFFACFF9CFF8CFF7CFA2
:10001200F6CFF5CF4FC0F3CFF2CFF1CFF0CFEFCF86
:10002200EECFEDCF1027E80364000A0001000010B4
:1000320000011000010000000000000000000000AC
:100042000000FC60DAF266B6BEE0FEE600000100E7
:10005200020038000A0004003A000000F894EE277B
:10006200ECBBF1E0FBBFEBBFE5BF8DE0A2E0BB273D
:10007200ED938A95E9F780E094E0A0E6ED9301978D
:10008200E9F7E0E5F0E085919591009761F0A5919F
:10009200B59105901590BF01F00105900D92019761
:1000A200E1F7FB01F0CFEFE5EDBFE4E0EEBFC0E624
:1000B200D1E035C0EA93FA93EFB7EA93C7D21BB106
:1000C2000CB1E12FEC7189F4E52D5394F0E0E05A84
:1000D200FE4F0083E8E0E51509F455247394E8E047
:1000E200E71519F47724689420F809911991E99198
:1000F200EFBFF991E99118951A937720F1F3E42D66
:100102004394F0E0E05AFE4F1081E8E0E41509F470
:100112004424F8947A947894E12F19910895D7D1D0
:100122007894E5D0E0918801F0918901309709F443
:10013200B2C0E0916C01F0916D01F9D131F4FBD1C3
:100142005F01CC24DD24FAD117C0E230A0E0FA0727
:1001520031F4AA24BB24EFD16F01F0D10DC0E330FA
:10016200A0E0FA0749F4AA24BB24CC24DD24E3D17D
:10017200E0937A01F0937B01E0916E01F0916F01BF
:10018200E330A0E0FA0709F081C0D5D1EA15FB05FA
:1001920031F4D1D1E0937C01F0937D0108C00A2CA7
:1001A2000B2829F4E0E0E0937C01E0937D01C3D1C8
:1001B200EC15FD0579F4C8D131F4BDD1E0937E018F
:1001C200F0937F0107C0309729F4E0E0E0937E01CD
:1001D200E0937F01A0917A01B0917B01119709F020
:1001E20055C0B2D111F4E1E003C0309719F4E0E058
:1001F200E0939001E0917201F0917301309731F434
:100202009AD1E0938201F093830107C090D129F43F
:10021200E0E0E0938201E0938301F0917401E0E079
:10022200DF01E0917601F0917701EA2BFB2B91D16E
:1002320095D199D118F0EFE0F7E28BD1E0917801F6
:10024200F0917901309731F4E0E0E0938601E09398
:1002520087011CC06CD111F46ED114C0E230A0E051
:10026200FA0719F4E2E0F0E00DC0E430A0E0FA078A
:1002720019F4E3E0F0E006C0E830A0E0FA0731F458
:10028200E4E0F0E0E0938601F0938701E0E0E093A0
:100292008801E0938901A0917C01B0917D011197C1
:1002A20011F465D122C0A0917E01B0917F01119716
:1002B200D1F4A0E8B1E0ED91FD913196FE93EE9379
:1002C200992039F454D158D118F0E1E09E2E59D139
:1002D20009C0E1E0E91531F441D149D04DD110F026
:1002E20099244FD102C03AD142D01BCFFFCF772001
:1002F200E9F1882081F400DFF0E0E0938C01F093D3
:100302008D01A0918C01B0918D01A03FE0E0BE076C
:1003120009F483942BC0E7E0E81598F0E82DF0E0AB
:100322003197ACE6B1E0EE0FFF1FEA0FFB1FFF9320
:10033200EF93E2DEAF91BF91F0E0ED93FC938394F3
:1003420015C0E8E0E81591F4D7DEF0E0E0938E0105
:10035200F0938F01A0918E01B0918F011D9729F426
:10036200EAD0E0938801F093890188240895BA9332
:10037200AA932B978BE0A0E0B0E0E4E4F0E069D12F
:1003820006D1E8EEF3E006D1E093680100D1E4E69D
:10039200F0E000D1E0936901FAD0EAE0F0E0FAD0AF
:1003A200E0936A01F4D0EAE0F0E04DD1E0936B0112
:1003B200DED0E8B3EC7FF4D0E07CF0E02CD127D1A2
:1003C200E029E8BBE5B3E07EEBD0EE73F0E0F59513
:1003D200E795E029E5BB6620D9F4A0919001A13010
:1003E20019F4E1E0E9D00FC0EBD019F4EFD0F3D06B
:1003F20009F005C0F3D0E0E0E2BBF2D004C0F6D0D1
:10040200119709F4979AE2B3E27EE2BB919A58C03F
:10041200E1E0E615D9F4EAD0129709F4979AD6D01A
:10042200E081E03011F0E7D00CC0CAD029F4CED080
:10043200D2D011F4E6D009F404C0D0D097989298A3
:10044200CFD0E2B3E47EE2BB929A3AC0E2E0E61594
:10045200D9F4CCD0139709F4979AB8D0E081E03060
:1004620011F0C9D00CC0ACD029F4B0D0B4D011F482
:10047200C8D009F404C0B2D097989398B1D0E2B32F
:10048200E87EE2BB939A1CC0E3E0E615C9F4AED065
:10049200149709F4979A9AD0E081E03011F0ABD02A
:1004A2000BC08ED029F492D096D011F4AAD009F4C0
:1004B20003C094D097989498E2B3E07FE2BB949AF9
:1004C2006394E4E0E61509F466242D960895E3E0CA
:1004D200E7BBE0E0E8BBEFE1E4BBE0E0E5BBEEEF69
:1004E200E1BBE0E0E2BBE3BFE2BFEFBDEEBDEDBDCD
:1004F200ECBDE7BDE6BDEBBDEABDE9BDE8BDE2BDD1
:10050200E5BDE4BDE3BDE9BFE5BFE2E0EBB9E0E98B
:10051200EAB9E6E8E0BDE0E0E0BDE0E1E9B9E0E843
:10052200E8B9E0E0E0BFE6B9EDB9E6BF0895E13031
:10053200A0E0FA070895E1E0F0E00895E0E0E0933A
:100542007A01E0937B010895E0917001F0917101CD
:10055200EECFE0938A01F0938B010895A0918A0176
:10056200B0918B010895A031E7E2BE070895E0E063
:10057200E8BBE5BBE2BB0895A0918001B091810187
:10058200F2CFE0E0E0938001E09381010895AB8532
:10059200BC85089545D0DF01EAE0F0E054D008952B
:1005A2000E2EE62DF0E0E859FE4FE081F0E0DE018C
:1005B200AE0FBF1FEC910895E5BBE0E0E8BB0895E4
:1005C200A0918201B091830111970895E62DF0E088
:1005D200E859FE4F0895A081A0300895E0E0ECCFE5
:1005E200AADFE0938401F09385010895A09186012A
:1005F200B09187010895E0E0E0938401E0938501E2
:100602000895E0918401F091850130970895F59560
:10061200E795F595E795F595E795F595E7950895AD
:100622000024112490E1AA0FBB1F001C111C0E1AFA
:100632001F0A18F40E0E1F1E01C0A1609A9599F7A9
:10064200FD01D0010895ECDFFD0108951A930A938C
:100652000895AC0FBD1F05900D928A95E1F708959C
:00000001FF
